:020000040000FA
:0600000000008A01B72D8B
:08000800F0000308F1000A08F2
:10001000F2008A0183120313083081070B115C2060
:1000200019205C2072088A0071088300F00E700E9F
:10003000090087013F200310F70DF71E0800741C0C
:100040002D28203084001930F8008413000884170C
:100050008000840AF80B25287410A0308400013039
:10006000F700F90803193628F9030319F414FA0BF9
:1000700008006430FA00FB08031DFB0308004B2056
:100080004B204B204B204B20043085000030850056
:100090007708870008000530F800000DF600F60D1F
:1000A000F60D0030F60D0318023885000138850082
:1000B000F80B5128840A08000408F3067306F306B7
:1000C00084000800F5186B2875186E28751D080047
:1000D0007220800608007220800408007220FF3A17
:1000E000800508003F0884000310840D840D8407F8
:1000F000203084074008840700308A003E088207C9
:10010000103408340434023401341930C100203072
:1001100084008009840AC10B892808001F30A000D0
:10012000A100A200A300A400A500A600A700A800AB
:10013000A900AA00AB00AC00AD00AE00AF00B0005B
:10014000B100B200B300B400B500B600B700B8000B
:1001500008001F30F5188000751880017519800699
:1001600008006220BD20BD20BD20BD200800622007
:10017000C120C120C120C1200800840A840A840A49
:10018000840A840AF518800475198006751880059C
:100190000800C001BF01B120C00AB120C00AB120CF
:1001A000C00AB120C00AB1200800C0017220A920F5
:1001B000840AA920840AA920840AA920840AA920E3
:1001C0000800BF017220A92005308407A92005304E
:1001D0008407A92005308407A92005308407A920B9
:1001E00008003330C500450884000008840A840AEA
:1001F000840A840A840A8000C50345081F3A031D47
:10020000F328A001A101A201A301A4010800253047
:10021000C500450884000008840384038403840324
:1002200084038000C50A4508393A031D0929B40131
:10023000B501B601B701B80108003730C50045085F
:1002400084000008840A8000C50345081F3A031D86
:100250001F29A001A501AA01AF01B40108002130A6
:10026000C50045088400000884038000C50A4508CD
:10027000393A031D3129A401A901AE01B301B80126
:1002800008001930C500203084008012800C840AD8
:10029000C50B452908001930C50020308400031023
:1002A000800D840AC50B4F2908006220C703073060
:1002B000470503198329C71D61293E0A3E19030119
:1002C000BE00461C68290430BE08031D3E03BE0064
:1002D000471E6E293F0A3F190301BF00C71E75293B
:1002E0000430BF08031D3F03BF00471F7B29400A9E
:1002F00040190301C000C71F82290430C008031D34
:100300004003C000552908002008C2003408A0009E
:100310003808B4002408B8004208A4002108C2002C
:100320002F08A1003708AF002908B7004208A9002C
:100330002208C2002A08A2003608AA002E08B60029
:100340004208AE002308C2002508A3003508A50016
:100350003308B5004208B3002608C2003008A600E2
:100360003208B0002808B2004208A8002708C200DE
:100370002B08A7003108AB002D08B1004208AD00E2
:1003800008000A248A01C600C61B122A461B022A3C
:1003900001308A00CF30460703188A0A8200C1293B
:1003A000E42AE72A892AAB2AB12AAE2A232ABB2AC1
:1003B000BB2ABB2A6E2AC62AC62AC62AB42AB72A4C
:1003C000B92A882B8A2B102B0E2B122B142B162BB1
:1003D000182B3F2A442A4A2A502A542A582A5C2A8F
:1003E000A92A0A2B3D2ADB2BE22BE92BF02BF72B3A
:1003F000EA2AED2A622AA12BA32BAC2BFE2BB12BD0
:10040000BC2BC92B5E2302308A000A304607031832
:100410008A0A8200DC2AD42AE02AD82A7C2B7F2B65
:10042000F72AFB2A0A248A01C700461B662AC61A35
:10043000702A460C0F39031D1F2A4C23C129FF3E89
:10044000031D252A4C236220C129FF3E031D2A2AB1
:100450005521C129FF3E031D2F2AF5151A2BFF3EFA
:10046000031D342AF5111A2BFF3E0319FF2AFF3E04
:100470000319042BFF3E0319922A8421C129342435
:100480007220A9203B24C1293424BF017220B1204D
:100490003B24C1293424C0017220B7203B24C12948
:1004A0003424C9203B24C1293424D5203B24C1292C
:1004B0003424E1203B24C1297220F41100050319E2
:1004C000F415C129F411051EF415C129C61A6823B3
:1004D00046081F39FD004708FC00C1297223C129C5
:1004E0005E234611460803197C2AFF3E03197F2A22
:1004F000FF3E0319832A112C47088000C1294708B1
:1005000012248000C129F41547080006031DF411C8
:10051000C129F41C892AF41074143D08F9007418D8
:100520008F2AC1296430FA004708FB00F411C7087C
:100530000319FB17FB080319C129051E972AC708D1
:100540000319FB17FB080319C129051A9F2AF41583
:10055000C1292D24C1290130F500C1290430F5003D
:10056000C1290230F500C12903018F20C1298E2045
:10057000C1298520C129460803393E3E8400043044
:100580008008031D00038000CF2AC12946080339D3
:100590003E3E8400800A0008053A03198001F415E4
:1005A0008008031DF411C1298003031DC129F02A0D
:1005B000800A031DC129F02AF415800BF411C1290A
:1005C000F415800FF411C129F41DC129F02AF41D7E
:1005D000F02AC129741EC129F02A741EF02AC129EB
:1005E0000A248A018039031D0A248A01C1290008CE
:1005F000C700F5151A2B0008C700F5111A2B643037
:10060000FA004708FB00C1296430FA0047081224A9
:10061000FB07C129FB08031DC129F02A1D21C1299F
:100620002F21C129F120C1290721C1294B21C1292D
:100630004121C1293424FF01203047023F39FE0007
:100640000310FE0DFE0DFE070318FF0A4230FE07E1
:100650000318FF0A0430FF070530C7000430F519FE
:10066000BF00F51DC001722048238A01F5188004DF
:1006700075198006FF3A75188005FE0A0319FF0AEE
:10068000F519BF03F51DC00AC70B332B3B24C12945
:100690007F088A007E0882004708BF000739C00033
:1006A000BF0CBF0C3F0C0739BF004708BE00460C0B
:1006B000BE0DBE0D3E0D0739BE00080046080739C5
:1006C000393E8400C60CC60C460C0739C60008002B
:1006D000430884007C088000840A7D088000040AA6
:1006E000C3000800430384000008FD0084030008E1
:1006F000FC000408C300080000088C23C12904087A
:10070000C7009823C5004708840045088000C12918
:10071000CD23C129D423C129C5004408840045083C
:100720008000C40A4408EB3AC9300319C400080029
:100730004408C93AEA30031D4403C4008400000899
:1007400008009823C1299823CE009823CF004E0893
:100750008C234F088C23C12998238C2345088C2394
:10076000C1299823CE009823CF004E088C234F0830
:100770008C234E088C23C1299823CE009823CF00C8
:100780009823D0004F088C234E088C2350088C23CC
:10079000C129982306248C23C1293E088C233F08B5
:1007A0008C2340088C2308009823C0009823BF00A6
:1007B0009823BE0008009823CD0098234D060624F8
:1007C0008C23C1299823CD0098234D0703248C2323
:1007D000C1299823CD0098234D0203248C23C129DD
:1007E0009823CD0098234D0506248C23C1299823F6
:1007F000CD0098234D0406248C23C1299823FF3A69
:1008000006248C23C129741203187416F4110319D9
:10081000F41508007D088A007C08FC0A0319FD0A0B
:100820008200112CCA000310C80CC90C031C1B2C1D
:10083000A130C806C9064808490403192D244908EF
:100840004807CB01CC01CC17CA0C0318CB07CB0C43
:10085000CC0C031C242C4B080800010803192D2C78
:10086000C900FF3AC80008003E08CE003F08CF008C
:100870004008D00008004E08BE004F08BF005008D6
:10088000C000080000340034003400340034043464
:1008900004340434003404340A340A340034003498
:1008A00000340A341F340A341F340A340F34143429
:1008B0000E3405341E3419341A3404340B34133412
:1008C000083414340D3412340D340C340C34043424
:1008D0000834003402340434043404340234083458
:1008E000043404340434083415340E341F340E3404
:1008F0001534043404341F340434043400340C3408
:100900000C3404340834003400341F340034003410
:100910000034003400340C340C3401340234043418
:10092000083410340E341334153419340E340434AE
:100930000C34043404340E341E34013406340834C8
:100940001F341E3401340E3401341E3406340A348C
:100950001F34023402341F3410341E3401341E3468
:10096000063408341E3411340E341F340234043477
:10097000083408340E3411340E3411340E340E346D
:1009800011340F3402340C340C340C3400340C3475
:100990000C340C3400340C34043408340234043481
:1009A00008340434023400341F3400341F3400345B
:1009B000083404340234043408340E34113402345C
:1009C000043404340E341534173410340E34043423
:1009D0000A341F34113411341E3409340E340934EE
:1009E0001E340F341034103410340F341E340934D4
:1009F000093409341E341F3410341E3410341F34AB
:100A00001F3410341E34103410340F3410341334A7
:100A100011340F34113411341F34113411340E34A5
:100A20000434043404340E340134013401341134F8
:100A30000E34133414341834143413341034103482
:100A4000103410341F3411341B3415341134113464
:100A5000113419341534133411340E341134113463
:100A600011340E341E3411341E34103410340C344E
:100A70001234163412340D341E3411341E3414342E
:100A800012340F3410340E3401341E341F34043445
:100A900004340434043411341134113411340E3458
:100AA0001134113411340A3404341134113415342E
:100AB0001B34113411340A3404340A34113411341F
:100AC0000A340434043404341F3402340434083443
:100AD0001F34073404340434043407341034083425
:100AE0000434023401341C340434043404341C341B
:100AF00004340A3411340034003400340034003437
:100B000000341F3487011930F800A0019F25F80B2D
:100B1000862D8316031300308F00831203130130D8
:100B2000F70087001930F8000130A0009F25F80B6E
:100B3000962D0310770D771A0130F700922D0230B1
:100B4000A00B00398500A000B225200801388500DF
:100B5000B2250430850077088700B2250030850073
:100B6000B2250800FF30FF3E031DB32D08006400CE
:100B70000730990083160313910170308F00033002
:100B80008100F83085003030950083120313203047
:100B900084008417800184138001840A841FC92D76
:100BA00083160313E030870083120313851E822D02
:100BB000A030F3000130F700F4140530FD00EC30F4
:100BC000FC00C930C400B930C3000130BD0008309A
:100BD0008100A0308B00C12921342B340234C6346B
:100BE0003E34E6346634A4340934A8341134503425
:100BF000E534FC34C534F33440340234C634C634EE
:100C000040340234CA34C03440340234CA34D63496
:100C100040340234CA345D3440340234CA348A3435
:100C200040340234C834343440340234CE34C63410
:100C300040340234CB34ED3440340234CC3470349C
:100C400040340234CD34083440340234CD340C34D2
:100C500040340234CD34103440340234CD34663460
:100C600040340234CF34773440340234CD34BF348E
:100C700040340234CE341A34C534FC34E63466349D
:100C8000E634C634EA34C034EA34D634EA345D3467
:100C9000EA348A34E8343434EE34C634EB34ED3498
:100CA000EC347034ED340834ED340C34ED3410345D
:100CB000ED346634EF347734ED34BF34EE341A3427
:100CC000C63440342234C63462340B34A63404347F
:100CD0000534A0345034E634B034A0344934E6341A
:100CE000B034A0344334E634B034A0345034E63465
:100CF000B034A0345234E634B034A0344F34E63447
:100D0000B034A0344A34E634B034A0344534E63448
:100D1000B034A0344334E634B034A0345434E63430
:100D2000B034A0345334E634B034A0344234E63422
:100D3000B034A0345934E634B034A0344A34E63404
:100D4000B034A0344F34E634B034A0345334E634F5
:100D5000B034A0344534E634B034143403340B34A6
:100D6000A43409340F34783403341734033417347B
:100D700003340F34A734023405347034033414348C
:100D800003341434A434233403340B34A43409342A
:100D90000534E634D034E7343E34E734A4340B343D
:100DA0000F345434833400348234043403348234B2
:100DB000C034823403348334013482344434033401
:100DC0008234803482340234823484348334023472
:100DD000033482344034823401348234C434833462
:100DE00003340334823400348334043403348234CF
:100DF000083483340C340334823410348334143490
:100E000003348234183483341C3403348234203461
:100E10008334243403348234603482342134833480
:100E200023348234E43403348234A03482342234D0
:100E30008234A4348334223403348234E034823460
:100E400023348334213482346434033483342034AF
:100E50008234243403348334183482341C3403340D
:100E600083341034823414340334833408348234A9
:100E70000C3454345434543403340B3482344134F9
:100E80008234C33403348234813482344234823431
:100E9000C2348234833403348234C13482344334E0
:100EA00003348234C93482344B3403348234D13431
:100EB0008234533403348234D93482345B3403347F
:100EC0008234E1348234633403348234A134823492
:100ED00062348234A3348234E234033482346134A1
:100EE0008234E3340334823459348234DB340334BF
:100EF000823451348234D3340334823449348234DA
:100F0000CB34033482348234033482348A3403345D
:100F100082349234033482349A3403348234A234D7
:100F200003340B34043407340934053407340334F0
:100F30004834C7349234043403340B34A0340434BA
:100F40005434E73492340B34A43401348234A23460
:100F5000E7349E3482346234E7349E34823463341E
:100F6000E7349E348234A334E7349E348234E3344D
:100F7000E7349E34A43401348234E234E7349E34BE
:100F80008234E134E7349E348234A134E7349E3431
:100F900082346134E7349E3482342134E7349E3421
:100FA000A434013482342234E7349E34823423342E
:100FB000E7349E3482342434E7349E3482346434FB
:100FC000E7349E348234A434E7349E34A4340134AC
:100FD0008234E434E7349E3483342434E7349E345A
:100FE00083342334E7349E3483342234E7349E340C
:100FF00083342134E7349E34A434013483342034E0
:10100000E7349E348234E034E7349E348234A034B2
:10101000E7349E3482346034E7349E3482342034A2
:10102000E7349E34A43414341634033416340334B1
:10103000233403341534053480344A3484340B3477
:101040008434133485340334843423348234923426
:101050000334153482349234033415340334153494
:101060000334153403340B3404340534A434093404
:101070008A340A348C340A340F3405340F3405347E
:101080008034A034843445348034993484344334F7
:10109000823458348234DC348034103484344D3417
:1010A0008034493484344B3483340B3482340934EF
:1010B0008034023484340D340334EA345A340F3427
:1010C00005348034A134843443348234603482342F
:1010D000E4348034183484344D34803451348434CE
:1010E0004B34833413348234113480340A348434DE
:1010F0000D348034C1348534433483340134823434
:1011000003340334EA345A340F3405348034203441
:1011100084344D348034593484344B3483341B3418
:10112000823419348034123484340D348034C93418
:101130008534433482340B348334093481340034AD
:10114000853445340334EA345A340F34053480345A
:10115000613484344B3483342334823421348034F6
:101160001A3484340D348034D13485344334823499
:101170001334833411348134083485344534803455
:10118000C134853443348234C0348234443403342B
:10119000EA345A348034223484340D3480345A345E
:1011A00084340B348334193482341B348134103446
:1011B000853445348034C934853443348234C8346A
:1011C00082344C3480348034843445340334EA34FB
:1011D0005A348034623484340B348334213482347E
:1011E000233481341834853445348034D134853403
:1011F00043348234D0348234543480348834843458
:1012000045348034813484344334823440348234ED
:10121000C4340334EA345A348134203485344534B8
:101220008034D934853443348234D83482345C34C5
:101230008034903484344534803489348434433465
:10124000823448348234CC348034003484344D3495
:101250000334EA345A348034E134853443348234FC
:10126000E0348234643480349834843445348034B7
:10127000913484344334823450348234D4348034CE
:10128000083484344D348034413484344B348334D2
:101290000334823401340334EA345A348034A034C1
:1012A000843445348034993484344334823458341B
:1012B0008234DC348034103484344D348034493406
:1012C00084344B3483340B34823409348034023414
:1012D00084340D340334EA345A348034A1348434F1
:1012E0004334823460348234E434803418348434B7
:1012F0004D348034513484344B3483341334823449
:10130000113480340A3484340D34803442348434CB
:101310000B3482340334833401340334EA345A34D2
:101320008034203484344D348034593484344B3404
:1013300083341B34823419348034123484340D34B1
:1013400080344A3484340B3482340B34833409348B
:1013500081340034853445340334EA345A348034DB
:10136000613484344B3483342334823421348034E4
:101370001A3484340D348034523484340B3482343F
:101380001334833411348134083485344534803443
:10139000C134853443348234C03482344434033419
:1013A000EA345A348034223484340D3480345A344C
:1013B00084340B3482341B34833419348134103434
:1013C000853445348034C934853443348234C83458
:1013D00082344C3480348034843445340334EA34E9
:1013E0005A348034623484340B348234233483346A
:1013F000213481341834853445348034D1348534F3
:1014000043348234D0348234543480348834843445
:1014100045348034813484344334823440348234DB
:10142000C4340334EA345A348134203485344534A6
:101430008034D934853443348234D83482345C34B3
:101440008034903484344534803489348434433453
:10145000823448348234CC348034003484344D3483
:101460000334EA345A348034E134853443348234EA
:10147000E0348234643480349834843445348034A5
:10148000913484344334823450348234D4348034BC
:10149000083484344D348034413484344B348334C0
:1014A00003348234013403340F3405342234C83415
:1014B0003C340B340F3405340B340F34033405340F
:1014C000A43423348234003483340034833420340D
:1014D0008334243482342434823404348334043412
:1014E0008234203403348234493482344B3482349D
:1014F000593482345B348234C9348234CB348234FC
:10150000D9348234DB3403348234923403340F34DC
:10151000C6346234A43432340F3405348234923405
:10152000033482348A3482349A348234523482349A
:10153000D2348234913482349334033480349234FC
:101540001A341B341C34823451348234D334823400
:1015500053348234D1348234893482348B348234AB
:101560004A348234CA348234993482349B3482348B
:101570005A348234DA3403348A340134C63462345F
:10158000A43407348A340F34A63404340F340534B9
:101590001734EA34D03403342234CA34C8340B3418
:1015A000AD340534AF34053407340B340F34043410
:1015B00005348A3407348C340634A4340934833433
:1015C00024340334A1340034A0340434EB34E13443
:1015D000A4340434EA34F634A1340134EB34D43482
:1015E000EA34F6342234CA34DD340B34EB340F34AD
:1015F000EB341834EB342534EB343634EB344B34E1
:10160000EB346634EB347D34EB349434EB34A9346E
:10161000EB34BA34EB34C734EB34D0340B3482348B
:1016200040348234013482340834EB34DA340B34FD
:101630008234103482344834823409348034803423
:1016400085344334EB34DA340B3482341834823446
:1016500050348234113480348834853443348034B7
:10166000C03485344434EB34DA340B3482342034DF
:10167000823458348234193480349034853443347D
:101680008034C8348534443481340034853445345E
:10169000EB34DA340B34833401348234C234823490
:1016A000833482344434813408348534453480347E
:1016B000D03485344434803498348534433482348F
:1016C000603482342134EB34DA340B348134023424
:1016D00085344334813409348534443481341034BE
:1016E000853445348034D834853444348034A0344F
:1016F00085344334EB34DA340B34833403348234AA
:10170000C43481340A34853443348134113485340B
:10171000443481341834853445348034E03485349D
:101720004434EB34DA340B348334043483340B34F0
:101730008234CC34813412348534433481341934C6
:10174000853444348134203485344534EB34DA3400
:101750000B3483340C34833413348234D4348134E2
:101760001A34853443348134213485344434EB34A1
:10177000DA340B348334143483341B348234DC3451
:101780008134223485344334EB34DA340B348334FB
:101790001C34833423348234E434EB34DA340B34B1
:1017A0008334243403340B34823400340434073457
:1017B00003340B340334B1340134023406340334BB
:1017C0000B3404340734083409340A34053407343C
:1017D00003344834CB34E1340B340F34A4340934AB
:1017E0000534823494340334823493348234533451
:1017F0008234D33482348B3482349B340334803447
:1018000092341A341B3482345A3482344A34823447
:10181000DA348234CA3403341434823494340334D2
:101820001434823494340334143482349434803441
:1018300000341F340434823400348234203483343E
:101840000034833420340334053414348234943423
:10185000803400341F3403340434823494348234AA
:10186000903403348234933482349034823450344C
:101870008234D034823488348234983403348234CD
:101880009234803490341A341B3482345834823485
:1018900048348234D8348234C834033405340F34A5
:1018A000823400348234203483340034833420344E
:1018B0000334153403341534033415340334153428
:1018C00003340F3482344C3482345C348234CC346C
:1018D0008234DC3403340F348234943403340B34D4
:1018E0008A3406348C3407340534A43409340F3474
:1018F0008034003484341D348434653485341534A4
:101900008434A53403340F348034403484341C349C
:1019100081342134843464348034C43485341434C0
:10192000803423348434A43403340F34803480343A
:1019300084341B3484345334843463348534233402
:1019400085341334843493348434A33484342B3472
:1019500003340F348034C03484341A34843454341F
:101960008434623485342434853412348434943499
:101970008434A23484342C3403340F34813400345E
:1019800084345534853425348434953484342D346A
:1019900003340F3481340134843454348034E434D7
:1019A0008534243480340334843494348034603473
:1019B00084342C3403340F3481340234843453346B
:1019C00085341334853423348434A33484349334F9
:1019D00084341B3484342B348434633403340F3420
:1019E00081340334843452348534143485342234BD
:1019F0008434A4348434923484341C3484342A34BB
:101A00008434643403340F342234CC3477340B34CC
:101A1000ED341434CD342734ED341434CD34513412
:101A2000ED341434CD343C340F340534AC34083444
:101A30006434A4340834643425346C348034103471
:101A4000A03401348A3404348C3406340B341C340E
:101A5000033419346034663425346E34B6340434B7
:101A60000234A034FF34B63400340234A0340134DC
:101A70002234CD3427340B341B3403341534603412
:101A8000653425346D34B53404340234A034FF3465
:101A9000B53400340234A03401342234CD343C3423
:101AA0000B341A34033415346034663425346E3400
:101AB000B63404340234A034FF34B6340034023473
:101AC000A03401342234CD3451340B34A4340A34DC
:101AD0000F3403348A3403348C34043405348334AF
:101AE0002434AB340334A4340A34ED348534A434C0
:101AF00005346434AC340C34643425346C34ED3443
:101B000092342234CD347F340B34B3340034023475
:101B10001F34B334013402341E34B334023402347B
:101B20001D340B34ED34A334ED34A334ED34A3343D
:101B3000ED34A334ED34B134ED34B134ED34B1349B
:101B4000ED34B1340B34B334003402341434B334D0
:101B5000013402341734B3340234023418340334F9
:101B60000B34B334003402341534B334013402344A
:101B70001634B33402340234193403340B340F34C2
:101B80008A3405348C340634A43401346434AC34DF
:101B90000734643425346C3480340034EE3401343A
:101BA0000D34EE340D340D34EE3401340D34EE3496
:101BB0000D340D34EE3401340E34EE340D340E3465
:101BC000EE3401340E34EE340D340E34EE34013480
:101BD0000934EE340D340934EE3401340934EE3472
:101BE0000D340934EE3401340A34EE340D340A3441
:101BF000EE3401340A34EE340D342234CD34C4349E
:101C00000B34053407340334043407340C34013402
:101C1000CE340134043408340B340534073403342F
:101C2000043407340834B53404340134CE340D346C
:101C30000C340B34A4340B348A340E34A634003400
:101C40000F340534A0340034EE348534EE343234AD
:101C50000734033416340734033416342234CE34B4
:101C600026340B34A9341034B13400340234EE3449
:101C70008E34B13401340234EE349334B13402344E
:101C80000234EE349834B13403340234EE349D34EB
:101C9000B13404340234EE349334B13405340234B4
:101CA000EE348E34B13406340234EE349834B13428
:101CB00007340234EE349D34B13408340234EE3447
:101CC000A234B13409340234EE34AB34B1340A34C2
:101CD0000234EE34B434B1340B340234EE34BD3457
:101CE000B1340C340234EE34A234B1340D34023445
:101CF000EE34AB34B1340E340234EE34B434B13497
:101D00000F340234EE34BD340B34AD340334553467
:101D1000AF3403345734073403340B34B53404344C
:101D200001340C340B34B734043401340E340B3426
:101D3000B5340034013408340B34B7340034013482
:101D40000A340B34B734043401340E34B53404345B
:101D500001340C340B34B534043401340C34B7344E
:101D6000003401340A340B34B534003401340834FF
:101D7000B734003401340A340B34B5340034013440
:101D80000834B734043401340E340B348A340A3442
:101D90000F340534A4340234A3340034CE34D034A8
:101DA000CF344734CE34D034A8341034B034003477
:101DB0000234EF342734B03401340234EF342E349B
:101DC000B03402340234EF343734B03403340234E4
:101DD000EF343E34B03404340234EF342734B034BA
:101DE00005340234EF342E34B03406340234EF3488
:101DF0003734B03407340234EF343E34B03408346E
:101E00000234EF342734B03409340234EF342E3442
:101E1000B0340A340234EF343734B0340B34023483
:101E2000EF343E34B0340C340234EF342734B03461
:101E30000D340234EF342E34B0340E340234EF3427
:101E40003734B0340F340234EF343E340B34AD3415
:101E50000534AE340534AF3403340B34AD340534BB
:101E6000AE340534AF340334573457340B34AD3407
:101E70000534AE340334AF3405340B34AD3405349B
:101E8000AE340334AF340534563456340B34B334E3
:101E900000340234EF345534B3347D340234CF345B
:101EA00061342234EF3447340B34EE34D4342034EC
:101EB0000234EF347234B3347D3402340B34CF3413
:101EC0005534EE34D43420340134EF346D34B3342B
:101ED000003402340B34CF34613404340734033417
:101EE00043340B3405340734033453340B348A340D
:101EF0000A348C340A340F3405342134A1340134CB
:101F0000CF348234B13401340234EF349D34B134EF
:101F10001A340234EF34A6342234CF3482340B34F2
:101F2000AE340534AF340534A43401346434AC34F5
:101F30000C34643425346C340B34A434643480346D
:101F400000341D340334EF34AF340B34A434643420
:101F5000813424341D340334EF34C2340B34EF3471
:101F60009034A0340434A534003420340134513486
:101F700020340134EF34D534B1341A3402340B3404
:101F8000CF34AF34EF349034A0340434A534043467
:101F900020340134413420340134EF34DF34B1349F
:101FA000013402340B34CF34C234043407340C34DB
:101FB0000534073403344834CF34D5340B34043477
:101FC000073408340534073403344834CF34DF345D
:021FD0000B34D0
:02400E00E43399
:1042000020004C004500440020004300750062007F
:1042100065002000560031002E0030002E003400D2
:10422000200043003300200061006E0069006D0033
:104230006100740069006F006E007300200031009F
:1042400035002D00300031002D00320030003100EB
:1042500031002000200070006900630070007200CF
:104260006F006A0065006300740073002E006F0029
:10427000720067002E0075006B00200020002800EF
:1042800063002900200032003000300039002D008A
:104290003200300031003100200050006500740011
:1042A0006500200047007200690066006600690032
:0842B000740068007300200097
:00000001FF
